:1000000000308A00B7290000831A0A289F00030ED7
:10001000A0000F2883129F00030EA000A0149F0EC3
:100020000408A1000C08A2000D08A30083128B1E77
:100030001B280B191C280900A0308100061A222851
:1000400000302328013093001508950A1308031D7A
:10005000512801301702031D51280E3015020318D4
:1000600035280530150203183828950194015128C8
:100070000A301502031C46280830140203184628CB
:100080001408940A0314960C9501512808301402A0
:10009000031851281408940A0310960C9501013096
:1000A0009900FB301502031C6128990101301A02E6
:1000B000031D5D2802309A00612803301A020319DB
:1000C0009A0108301402031D6928093094001608AB
:1000D0009800130897000B112108840022088C0057
:1000E00023088D00200E830083121F0EA018831694
:1000F000090028080319892801308D008C018C0B18
:100100007F288D0B7E284A308C008C0B8528A80B0D
:100110007C28003486110000000000000000000070
:10012000861506308C008C0B932886110000000089
:10013000000000000000861506308C008C0B9E2805
:100140008611000000000000000000008615063047
:100150008C008C0BA9288611000000000000000014
:100160000000861506308C008C0BB4288611000028
:100170000000000000000000861506308C008C0B8B
:10018000BF282708031DCA2842308C008C0BC628C4
:100190000000EF2801302702031DD6280130A800F7
:1001A000792021308C008C0BD328EF2802302702D5
:1001B000031DE82853308C008C0BDC2853308C0056
:1001C0008C0BE02810308C008C0BE4280000EF280A
:1001D00003302702031DEF280230A80079200034E5
:1001E0008B13A7018A20260801398C0001300C02EC
:1001F000031DFE280130A7008A2001290230A70034
:100200008A20260802398C0003108C0C0C088C0004
:1002100001300C02031D10290130A7008A20132988
:100220000230A7008A20260804398C008C0C8C0C24
:100230003F308C050C088C0001300C02031D242972
:100240000130A7008A2027290230A7008A2026082B
:1002500008398C008C0C8C0C8C0C1F308C050C0815
:100260008C0001300C02031D39290130A7008A20BF
:100270003C290230A7008A20260810398C008C0EF9
:100280000F308C050C088C0001300C02031D4C292A
:100290000130A7008A204F290230A7008A202608B3
:1002A00020398C008C0E8C0C07308C050C088C00CF
:1002B00001300C02031D60290130A7008A20632948
:1002C0000230A7008A20260840398C008C0E8C0C46
:1002D0008C0C03308C050C088C0001300C02031DC3
:1002E00075290130A7008A2078290230A7008A20CA
:1002F000260880398C008C0E8C0C8C0C8C0C0130F8
:100300008C050C088C0001300C02031D8B29013078
:10031000A7008A208E290230A7008A200330A70078
:100320008A208B17003401308E000130A600F020A7
:10033000A401043024020318AD290F3024078400DF
:100340000008A5002508A600F0200F30240784002F
:1003500000088E062408A40A992901300E02031D04
:10036000B32902308E000E08A600F020FA2984017D
:10037000940195010130970099019A0109309E007E
:100380008B133030660008308C008C1DCF2907306D
:100390008101813084000008C0390F38800064007A
:1003A000813084000008C0390C0480008B168B1744
:1003B000890183160814831208088F000130890010
:1003C00083160814831208089000023089008316EF
:1003D0000814831208089100920106110230A4004B
:1003E000FA30A8007920A40BF02906151908031D7E
:1003F000FB2993294A2A09301402031D4A2A940131
:100400001B08031D0C2A01301802031D0C2A1808B2
:100410009C0001309B004A2A01301B02031D172A51
:1004200018089D0018089C0602309B004A2A0230DA
:100430001B02031D492A01301C02031D212A023020
:100440009C001C081802031D472A1D081E02031DDC
:10045000452A1A08031D332A1D089200990101300C
:100460009A000611442A01301A02031D392A990103
:10047000442A02301A02031D432A920199010330D3
:100480009A000615442A9901472A1D089E009B01DF
:100490004A2A9B01F6296300FF3FFF3FFF3FFF3FD2
:1004A000FF3FFF3FFF3FFF3FFF3FFF3FFF3FFF3F5C
:1004B000FF3FFF3FFF3FFF3FFF3FFF3FFF3FFF3F4C
:1004C000FF3FFF3FFF3FFF3FFF3FFF3FFF3FFF3F3C
:1004D000FF3FFF3FFF3FFF3FFF3FFF3FFF3FFF3F2C
:00000001FF
